:020000040000FA
:020000003A289C
:08000800A000030EA100831209
:100010008B1C32288B102D181428AD1C322864300C
:10002000010203183128182800001628172818285C
:1000300019281A281B281C281D281E281F282D10A7
:10004000AD14A610031005190314A80DA70DA60DD5
:10005000AC0B32282D152808AB002708AA0026086B
:10006000A900AD1081010B11210E8300A00E200EFE
:02007000090085
:0C007400203084008001840A6030040207
:10008000031C3C281230AC003A143D140730C80061
:100090005A30C900CA008316FF23900083128316CA
:1000A0000512851287100712871187120711051490
:1000B00085140515851507148312850187010730FE
:1000C000990011309F00103083169F00831210306A
:1000D000831691008312C830831681008312313059
:1000E0009000003083168C00831210308B00831632
:1000F00010309B001C141A088312D2005218871467
:10010000831600309B001C141A088312B3008B174F
:1001100033082F3C031CB301E6202D192E22BC0806
:10012000031D70234B182D231E303D05031DA228EF
:100130003A18FC20BA180C213A191A213A1BD0217E
:10014000BA1BDC2150080E02031885127C303A05D8
:10015000031DB628BC08031DB628BD08031DB6281C
:1001600051080E0203180716031887118F08031988
:100170008C288F013C303A05031D85161E303D0545
:10018000031DEA23BC08031DCB28FE303A05031DDE
:100190000712031D8715E6210A2218303A05031DB0
:1001A000DE20BA1935213A1A8221C80B8C28073073
:1001B000C800BA1E8C28DE20B6218C289F14350377
:1001C000B6009F18E1281E08B500080064002D182D
:1001D00008000B1D08000B11AD102D141230AC00DF
:1001E000051DF7282E1483160113831208002E1004
:1001F00083160117831208008712B701B801D001D6
:10020000D101BB0111235314B91F0800B9131430D5
:10021000C600BA01BA140800C60B08001430C600A4
:10022000D10F0800D1030630C600FF30C700BA0165
:100230003A1508008716FF30D000C70B0800C60B20
:10024000080001303B18B9003030051A013E831612
:100250009B001C141A088312043ED0001930C600FB
:10026000FF30C700BA01BA150800AA303502031CD6
:100270004029D31C43295315D40F4329D4034329C0
:10028000D4015318D314C830350203184C29143044
:10029000B802031C512908001430B80703185A2962
:1002A0000800B801C70B0800C60B0800B901BA0165
:1002B0003A140800B801531D6829D3010030541ABC
:1002C000013ED41A023E541B073ED41B103ED500FB
:1002D00001303B18B9000130390220300319103EBB
:1002E000051A013E83169B001C141A088312163C43
:1002F000003C5507D0000C30C600FF30C700BA01E3
:100300003A160800C8303502031C8B291430B80295
:10031000031C902908001430B80703189929080015
:10032000B801C70B0800C60B0800B901BA013A149E
:100330000800051A2023051E2623B90BAF293030EB
:10034000051A013E83169B001C141A0883121A3CDE
:10035000003C5507D000BA01BA16B70108001930A1
:10036000C600FF30C700BA01BA15080035083602CA
:10037000031CBF294130B702031CC42908005830B0
:10038000B7070318C6290800B7010800B70185128E
:10039000D0016430C600FF30C700BA013A17080028
:1003A0000715C70B0800C60B080007111A231430E5
:1003B000C600BA01BA170800C60B08001430C60000
:1003C000D10B0800B901BA013A1408000518ED294B
:1003D0001930C9070318F22908000A30C902031CA2
:1003E000012A0800FF30C9003A1C08004B14643091
:1003F0004A02031808004B10CB14C030B900051690
:100400000800C9014B10CB133D10CB1C0800CB01D9
:100410003B1408008518112A1930CA070318162A38
:1004200008000A30CA02031C252A0800FF30CA004F
:100430003A1C08004B1464304902031808004B10A2
:100440004B15C030B90005120800CA014B10CB1380
:100450003D104B1D0800CB013B1408002D112E1C34
:10046000362A29090339A900AA09AB093C083D0429
:100470000319452A2B1CAD132B1C0800AD1B0800CB
:100480002A180800AD173C18432B0430C300003075
:10049000C4008B1383162030440743079B001C14B1
:1004A0001A088312A400A500C030A50683161030D8
:1004B000440743079B001C141A088312A3008316E9
:1004C0000030440743079B001C141A088312A20043
:1004D0008B1722082902031D032B23082A02031D60
:1004E000032B24082B02031DC42AC408031DA12AC0
:1004F00004304302031D802A87145214D217032BA1
:1005000005304302031D8F2AFE303A05031DF42AED
:10051000BD08031DFE2A8130B90005120800FE3017
:100520003A05031D080006304302031D9B2A98303C
:10053000B9000512080007304302031DA12A051265
:100540000800FE303A05031D08008B138316303077
:10055000440743079B001C141A088312B4008B172E
:1005600033083402031C303EB40018303402031840
:10057000B42A031C183EB400B40803190800051E71
:10058000183CB900B9170800C408031D032B25083F
:100590002B02031D032B04304302031DD32A8710B3
:1005A0005210D217032B05304302031DE22AFE30FE
:1005B0003A05031DF42ABD08031DF52A8130B90050
:1005C00005160800FE303A05031D080006304302F8
:1005D000031DEE2A9830B9000516080007304302C3
:1005E000031D032B0516080008000530D007F53061
:1005F0005002031C0800F530D00008000530D0027E
:10060000031CD0010800C30AC31D082BBC18432BD0
:10061000431E492AC408031D0800C3014030C4001A
:10062000492AD21F0800D2131030BF005208BE0062
:10063000902308000030BF003308BE00902308005C
:10064000B30A33082F3C031CB3010800B30333087B
:100650002F3C2F30031CB3000800CB1B0800CB1726
:10066000BD08031DA32BBC08031D602B850187015A
:10067000071687153C14BC101430B2000430C100BA
:100680000030C20008008B13303042074107BF0022
:100690003308BE009023203042074107BF002B08DB
:1006A000BE009023103042074107BF002A08BE0059
:1006B0009023003042074107BF002908BE00902365
:1006C0000712C10AB0011430B200411E0800C2086E
:1006D000031DBC10031D0800C1014030C20008000A
:1006E0006400B10B0800321E0712B20B0800B008FC
:1006F00003197D2B0716B0038D2B4108B00008307D
:100700004102031C872BB00087113C10BC14B00AB7
:10071000871D8D2B03304102B0001430B200080059
:100720008B133E0883161C159A003F089B0055301A
:100730009D00AA309D009C1464009C189C2B1C11E9
:1007400083128B1708000310BD0DBD1CAF2B831641
:1007500020309B001C141A088312D00005123D1D86
:10076000BE2B2030BF005008BE00902383163030CF
:100770009B001C141A088312D0000512BD1DCD2B3E
:100780003030BF005008BE009023831631309B00EC
:100790001C141A088312D00005163D1EDC2B3130C4
:1007A000BF005008BE009023831621309B001C140C
:1007B0001A088312D0000516BD1EE92B2130BF0098
:1007C0005008BE009023D001BD010512B901BA0145
:1007D0003A14080087168516DE200712C830350245
:1007E000031C07168711AA303502031C8715373002
:0807F0003502031C071208008A
:084000000B00010004000400A4
:02400E00CC01E3
:104200000000FF00FF00FF000000000000000000B1
:104210000300030003000300030003000300030086
:104220000100FF00FF00FF00C800C800C800C80070
:10423000C800C800C800C800C800C800C800C8003E
:10424000F500F500FF00FF00C300F300CF00FF0002
:104250000300C3003300F3000F00CF003F00FF0056
:1042600078007800FF00FF00FF00FF00FF00FF0064
:104270000000010002000300040005000600070022
:10428000020002000200020002000200020002001E
:10429000000000000000000000000000000000001E
:1042A000C800C800C800C800C800C800C800C800CE
:1042B00088008800880088008800880088008800BE
:1042C0000300C3003300F3000F00CF003F00FF00E6
:1042D0000300C3003300F3000F00CF003F00FF00D6
:1042E000080009000A000B000C000D000E000F0072
:1042F0001000110012001300140015001600170022
:00000001FF
